:1000000019C023C118951895189518951895189525
:100010001895189518951895189518951895189578
:100020001895189518951895189518951895189568
:10003000189518958FEF8DBFC0EEE0EE4E2E84E040
:100040008EBFD4E0F4E05F2EEEEFF3E0A0E0B1E08D
:1000500088278D933197E9F784B7082E877F84BF6F
:100060008FE18093600087E08093600039DB662435
:1000700088E78AB986EC87B98FE384B980E08BB9C9
:1000800080E088B980EC85B95A9A5E9A78940EDB44
:100090008CE06EDBE2E1F9E101DBE1E0F0E017DBAF
:1000A00003DBE2E2F9E1FADA84EF91E08DDBE8E2EA
:1000B000F9E1F4DA84EF91E087DBEEE2F9E1EEDAE0
:1000C0008AEF90E081DBE0E3F9E1E8DA8AEF90E0A3
:1000D0007BDBE2E3F9E1E2DA8AEF90E075DBE4E36F
:1000E000F9E1DCDA8AEF90E06FDBE6E3F9E1D6DAFA
:1000F0008AEF90E069DBE8E3F9E1D0DA8AEF90E09B
:1001000063DBEAE3F9E1CADA8AEF90E05DDBECE376
:10011000F9E1C4DAE3E0F0E0DADAC8DAEEE3F9E1D3
:10012000BDDAC2DAEEE3F9E1B9DAE2E0F0E0CFDA23
:10013000BDDAEEE4F9E1B2DAB7DAEEE5F9E1AEDA2A
:10014000E2E0F0E0C4DAB2DAA3E2B0E00C9106FB40
:1001500081E00EF080E08F93A3E2B0E00C9107FB0A
:1001600081E00EF080E09F918923882309F403C089
:1001700081E080931101A3E2B0E00C9106FB81E0E5
:100180000EF480E08F93A3E2B0E00C9107FB81E0D6
:100190000EF080E09F918923882309F403C082E058
:1001A00080931101A3E2B0E00C9106FB81E00EF018
:1001B00080E08F93A3E2B0E00C9107FB81E00EF4A6
:1001C00080E09F918923882309F403C083E0809312
:1001D0001101A3E2B0E00C9106FB81E00EF480E097
:1001E0008F93A3E2B0E00C9107FB81E00EF480E076
:1001F0009F918923882309F403C084E0809311012F
:1002000000911101013009F003C0EEE6F9E146DA90
:1002100000911101023009F003C0ECE7F9E13EDA88
:1002200000911101033009F003C0EEE8F9E136DA7C
:1002300000911101043009F003C0E0EAF9E12EDA7F
:10024000E89A85E083BF88957FCFE898EDEFF1E0ED
:10025000ABE0B1E091E056DB00910B010E3C08F001
:1002600028C024DA00911101013009F003C0E2EB4B
:10027000F9E114DA00911101023009F003C0E4EC55
:10028000F9E10CDA00911101033009F003C0E6ED49
:10029000F9E104DA00911101043009F003C0E8EE3D
:1002A000F9E1FCD901DAE2E1F9E1F8D985E083BFAF
:1002B000889584E690E088DAA3E2B0E00C9106FB32
:1002C00081E00EF080E08F93A3E2B0E00C9107FB99
:1002D00081E00EF080E09F918923882309F403C018
:1002E00081E080931101A3E2B0E00C9106FB81E074
:1002F0000EF480E08F93A3E2B0E00C9107FB81E065
:100300000EF080E09F918923882309F403C082E0E6
:1003100080931101A3E2B0E00C9106FB81E00EF0A6
:1003200080E08F93A3E2B0E00C9107FB81E00EF434
:1003300080E09F918923882309F403C083E08093A0
:100340001101A3E2B0E00C9106FB81E00EF480E025
:100350008F93A3E2B0E00C9107FB81E00EF480E004
:100360009F918923882309F403C084E080931101BD
:10037000499901C0A3D34A9919C05E9888E290E0D8
:1003800023DA419A429A8AE090E01EDA42988AE0A3
:1003900090E01ADA4198429A8AE090E015DA4298A1
:1003A000309901C07ED2309B01C065D41895089564
:1003B0007DD900911101013009F003C0EAEFF9E1A4
:1003C0006DD900911101023009F003C0E8E0FAE1B3
:1003D00065D900911101033009F003C0E6E1FAE1AB
:1003E0005DD900911101043009F003C0E6E2FAE1A1
:1003F00055D9EEEFF1E0ADE0B1E081DA00910D0109
:1004000041E0040FAAE0B1E00C93A9E2B0E00C9146
:1004100000FB81E00EF080E08F93A6E2B0E00C914B
:1004200005FB81E00EF080E09F918923882309F489
:1004300003C088E080931001A9E2B0E00C9100FBBA
:1004400081E00EF480E08F93A6E2B0E00C9105FB12
:1004500081E00EF080E09F918923882309F403C096
:1004600080E180931001A9E2B0E00C9100FB81E0F3
:100470000EF080E08F93A6E2B0E00C9105FB81E0E6
:100480000EF480E09F918923882309F403C088E15A
:1004900080931001A9E2B0E00C9100FB81E00EF422
:1004A00080E08F93A6E2B0E00C9105FB81E00EF4B2
:1004B00080E09F918923882309F403C080E2809320
:1004C00010014091100100910A01041710F009F089
:1004D00001C070C080E080930D01EEEFF1E0ADE06F
:1004E000B1E07BE7FBD95E9A8AEF8093050184E057
:1004F0008093070184D8DAD800911101013009F006
:1005000003C0E8E3FAE1CAD800911101023009F012
:1005100003C0E6E4FAE1C2D800911101033009F00A
:1005200003C0E4E5FAE1BAD800911101043009F002
:1005300003C0E4E6FAE1B2D8009110010A3008F0F5
:1005400003C0E0E3F9E1AAD8A8ECB4E0E0E1F1E00F
:1005500075D99CD8A9D800911101013009F003C0C8
:10056000E2E7FAE19BD800911101023009F003C0E3
:10057000E4E8FAE193D800911101033009F003C0D7
:10058000E6E9FAE18BD800911101043009F003C0CB
:10059000E6EAFAE183D88AEF8093050184E080934C
:1005A00007012DD84A9901C0FDCF80D884E690E09C
:1005B0000BD9089579D85E9A00911101013009F0A4
:1005C00003C0EEE6F9E16AD800911101023009F0AA
:1005D00003C0ECE7F9E162D800911101033009F0A2
:1005E00003C0E6EBFAE15AD800911101043009F09A
:1005F00003C0E6ECFAE152D88AEF8093050180E06F
:1006000080930701FCD74A9901C0FDCFA9E2B0E071
:100610008C9182FBDEF7A9E2B0E08C9182FBDEF3E5
:100620005E9888E290E0D0D8419A429A8AE090E0C1
:10063000CBD842988AE090E0C7D84198429A8AE0A5
:1006400090E0C2D8429881E08093010100910101BD
:100650000F3010F009F083C000910101023009F061
:100660002AC0009100010F3F09F025C01FD800915A
:100670001101013009F003C0E6EDFAE10FD8009155
:100680001101023009F003C0E4EEFAE107D800914D
:100690001101033009F003C0E4EFFAE1FFD7009144
:1006A0001101043009F003C0E4E0FBE1F7D7E2E018
:1006B000F0E00DD86FC780E08093000180E0809368
:1006C000020100910201073010F009F01FC0A0E004
:1006D000B1E00C9142E0049F0C9200910001A6E26F
:1006E000B0E08C9183FB882780F9482F040FA0E0AD
:1006F000B1E00C93429A8AE090E066D84298A2E07A
:10070000B1E08C918F5F8C9308F4DBCFAAE0B1E06D
:100710000D9111274FE050E066D8A3E0B1E00D93B2
:100720001C93A3E0B1E00D911C91A1E0B1E04D91CB
:100730005527040F151FA3E0B1E00D931C93A3E010
:10074000B1E0ED91FC91A0E0B1E091E07BE7C9D888
:10075000A1E0B1E08C918F5F8C9308F477CFEEEF3E
:10076000F1E0AAE0B1E07BE7B9D884E690E02CD8CC
:100770005E9A8AEF8093050181E08093070196D706
:1007800000911101013009F003C0E4E1FBE186D7DB
:1007900000911101023009F003C0EEE1FBE17ED7C8
:1007A00000911101033009F003C0E8E2FBE176D7C4
:1007B00000911101043009F003C0E2E3FBE16ED7C0
:1007C00000910A010A3008F003C0E0E3F9E166D7BE
:1007D000A8ECB4E0EAE0F1E031D858D7009111017B
:1007E000013009F003C0ECE3FBE158D7009111019F
:1007F000023009F003C0E2E4FBE150D7009111019F
:10080000033009F003C0E8E4FBE148D7009111018F
:10081000043009F003C0EEE4FBE140D70091100181
:100820000A3008F003C0E0E3F9E138D7A8ECB4E0FF
:10083000E0E1F1E003D82AD737D700911101013068
:1008400009F003C0E4E5FBE129D700911101023072
:1008500009F003C0E0E6FBE121D70091110103306C
:1008600009F003C0ECE6FBE119D700911101043057
:1008700009F003C0EAE7FBE111D7C1D64A9901C0EC
:10088000FDCF14D7E1E0F0E022D786E9809305019F
:1008900000910A0141E0041BA7E0B1E00C93AFD640
:1008A000089504D700911101013009F003C0E6E872
:1008B000FBE1F4D600911101023009F003C0E2E936
:1008C000FBE1ECD600911101033009F003C0EEE921
:1008D000FBE1E4D600911101043009F003C0EAEA1B
:1008E000FBE1DCD6E1D600911101013009F003C033
:1008F000E6EBFBE1D3D600911101023009F003C011
:10090000E4ECFBE1CBD600911101033009F003C008
:10091000E4EDFBE1C3D600911101043009F003C0FE
:10092000E2EEFBE1BBD684EF91E04ED781E080930D
:100930000101009101010F3010F009F06AC000912F
:100940000101023009F02AC0009100010F3F09F0B7
:1009500025C0ACD600911101013009F003C0E6EDCD
:10096000FAE19CD600911101023009F003C0E2EFD8
:10097000FBE194D600911101033009F003C0E4EFCC
:10098000FAE18CD600911101043009F003C0E4E0D3
:10099000FBE184D6E2E0F0E09AD6FCC580E08093EB
:1009A000000180E08093020100910201073010F005
:1009B00009F01FC0A0E0B1E00C9142E0049F0C924E
:1009C00000910001A6E2B0E08C9183FB882780F9BA
:1009D000482F040FA0E0B1E00C93429A8AE090E027
:1009E000F3D64298A2E0B1E08C918F5F8C9308F42B
:1009F000DBCFA1E0B1E0EC91FF27A0E0B1E091E016
:100A00007BE76FD7A1E0B1E08C918F5F8C9308F406
:100A100090CF84E690E0D8D65E9A8AEF8093050165
:100A200081E08093070142D600911101013009F065
:100A300003C0E6EBFBE132D600911101023009F070
:100A400003C0E2E0FCE12AD600911101033009F075
:100A500003C0E4EDFBE122D600911101043009F05E
:100A600003C0E2EEFBE11AD61FD60091110101305E
:100A700009F003C0E4E5FBE111D600911101023059
:100A800009F003C0E0E6FBE109D600911101033053
:100A900009F003C0ECE6FBE101D60091110104303E
:100AA00009F003C0E2E1FCE1F9D5A9D54A9901C0FA
:100AB000FDCF309901C0FACFF9D50895F7D500914F
:100AC0001101013009F003C0E0E2FCE1E7D500913B
:100AD0001101023009F003C0E0E3FCE1DFD5009131
:100AE0001101033009F003C0E0E4FCE1D7D5009127
:100AF0001101043009F003C0E0E5FCE1CFD5D4D505
:100B000000911101013009F003C0E0E6FCE1C6D517
:100B100000911101023009F003C0E0E7FCE1BED50D
:100B200000911101033009F003C0EEE7FCE1B6D5F6
:100B300000911101043009F003C0EEE8FCE1AED5EC
:100B400081E080930F0180E190E0A8E0B1E08D9317
:100B50009C93A8E0B1E00D911C910C3F51E015076A
:100B600010F009F02AC000910F01083F09F003C0FE
:100B700080E38093070100910701003309F005C06D
:100B800080910F01815080930F0100910701003384
:100B900009F405C0AFE0B1E08C918F5F8C93A8E0C1
:100BA000B1E0ED91FC91AFE0B1E091E07BE799D647
:100BB000A8E0B1E043D508F4CCCF80E080930D01EC
:100BC000EEEFF1E0ADE0B1E07BE788D684E690E0BF
:100BD000FBD55E9A8AEF8093050182E0809307013E
:100BE00065D500911101013009F003C0ECE9FCE189
:100BF00055D500911101023009F003C0ECEAFCE187
:100C00004DD500911101033009F003C0EEEBFCE17A
:100C100045D500911101043009F003C0EEECFCE170
:100C20003DD542D500911101013009F003C0EEED30
:100C3000FCE134D500911101023009F003C0E0EF6E
:100C4000FCE12CD500911101033009F003C0E2E072
:100C5000FDE124D500911101043009F003C0E4E165
:100C6000FDE11CD5CCD44A9901C0FDCF499901C002
:100C7000FACF1CD5089580E080930F0117D58FE738
:100C800011E023D500911101013009F003C0E6E223
:100C9000FDE104D500911101023009F003C0E4E345
:100CA000FDE1FCD400911101033009F003C0E2E43E
:100CB000FDE1F4D400911101043009F003C0EEE429
:100CC000FDE1ECD484EF91E07FD581E080930101D8
:100CD000009101010F3010F009F0E5C380E080932E
:100CE000000180E08093020100910201073010F0C2
:100CF00009F01CC0A0E0B1E00C9142E0049F0C920E
:100D000000910001A6E2B0E08C9183FB882780F976
:100D1000482F040FA0E0B1E00C93429A4298A2E061
:100D2000B1E08C918F5F8C9308F4DECFA1E0B1E04D
:100D3000EC91FF27A6E0B1E091E0E4D540910601F7
:100D400000910001041709F401C006C0AFE0B1E052
:100D50008C918F5F8C93A0C3A1E0B1E00D9111271E
:100D60004FE050E0040F151FA3E0B1E00D931C937A
:100D7000A3E0B1E0ED91FC91A6E0B1E091E0C2D535
:100D80004091060100910001041709F401C001C05F
:100D900083C3A1E0B1E00D9111274EE150E0040FB3
:100DA000151FA3E0B1E00D931C93A3E0B1E0ED911A
:100DB000FC91A6E0B1E091E0A5D54091060100913B
:100DC0000001041709F401C001C066C3A1E0B1E04D
:100DD0000D9111274DE250E0040F151FA3E0B1E083
:100DE0000D931C93A3E0B1E0ED91FC91A6E0B1E07E
:100DF00091E088D54091060100910001041709F4A3
:100E000001C001C049C3A1E0B1E00D9111274CE33D
:100E100050E0040F151FA3E0B1E00D931C93A3E075
:100E2000B1E0ED91FC91A6E0B1E091E06BD540918D
:100E3000060100910001041709F401C001C02CC390
:100E4000A1E0B1E00D9111274BE450E0040F151F14
:100E5000A3E0B1E00D931C93A3E0B1E0ED91FC9110
:100E6000A6E0B1E091E04ED540910601009100016D
:100E7000041709F401C001C00FC3A1E0B1E00D9156
:100E800011274AE550E0040F151FA3E0B1E00D93D0
:100E90001C93A3E0B1E0ED91FC91A6E0B1E091E0FC
:100EA00031D54091060100910001041709F401C0F9
:100EB00001C0F2C2A1E0B1E00D91112749E650E076
:100EC000040F151FA3E0B1E00D931C93A3E0B1E064
:100ED000ED91FC91A6E0B1E091E014D540910601BE
:100EE00000910001041709F401C001C0D5C2A1E0BE
:100EF000B1E00D91112748E750E0040F151FA3E062
:100F0000B1E00D931C93A3E0B1E0ED91FC91A6E05C
:100F1000B1E091E0F7D4409106010091000104177F
:100F200009F401C001C0B8C2A1E0B1E00D911127E0
:100F300047E850E0040F151FA3E0B1E00D931C93A8
:100F4000A3E0B1E0ED91FC91A6E0B1E091E0DAD44C
:100F50004091060100910001041709F401C001C08D
:100F60009BC2A1E0B1E00D91112746E950E0040FCA
:100F7000151FA3E0B1E00D931C93A3E0B1E0ED9148
:100F8000FC91A6E0B1E091E0BDD440910601009152
:100F90000001041709F401C001C07EC2A1E0B1E064
:100FA0000D91112745EA50E0040F151FA3E0B1E0B1
:100FB0000D931C93A3E0B1E0ED91FC91A6E0B1E0AC
:100FC00091E0A0D44091060100910001041709F4BA
:100FD00001C001C061C2A1E0B1E00D91112744EB55
:100FE00050E0040F151FA3E0B1E00D931C93A3E0A4
:100FF000B1E0ED91FC91A6E0B1E091E083D44091A5
:10100000060100910001041709F401C001C044C2A7
:10101000A1E0B1E00D91112743EC50E0040F151F42
:10102000A3E0B1E00D931C93A3E0B1E0ED91FC913E
:10103000A6E0B1E091E066D4409106010091000184
:10104000041709F401C001C027C2A1E0B1E00D916D
:10105000112742ED50E0040F151FA3E0B1E00D93FE
:101060001C93A3E0B1E0ED91FC91A6E0B1E091E02A
:1010700049D44091060100910001041709F401C010
:1010800001C00AC2A1E0B1E00D91112741EE50E08C
:10109000040F151FA3E0B1E00D931C93A3E0B1E092
:1010A000ED91FC91A6E0B1E091E02CD440910601D5
:1010B00000910001041709F401C001C0EDC1A1E0D5
:1010C000B1E00D91112740EF50E0040F151FA3E090
:1010D000B1E00D931C93A3E0B1E0ED91FC91A6E08B
:1010E000B1E091E00FD44091060100910001041796
:1010F00009F401C001C0D0C1A1E0B1E00D911127F8
:101100004FEF50E0040F151FA3E0B1E00D931C93C7
:10111000A3E0B1E0ED91FC91A6E0B1E091E0F2D363
:101120004091060100910001041709F401C001C0BB
:10113000B3C1A1E0B1E00D9111274EE051E0040FE1
:10114000151FA3E0B1E00D931C93A3E0B1E0ED9176
:10115000FC91A6E0B1E091E0D5D340910601009169
:101160000001041709F401C001C096C1A1E0B1E07B
:101170000D9111274DE151E0040F151FA3E0B1E0DF
:101180000D931C93A3E0B1E0ED91FC91A6E0B1E0DA
:1011900091E0B8D34091060100910001041709F4D1
:1011A00001C001C079C1A1E0B1E00D9111274CE26D
:1011B00051E0040F151FA3E0B1E00D931C93A3E0D1
:1011C000B1E0ED91FC91A6E0B1E091E09BD34091BC
:1011D000060100910001041709F401C001C05CC1BF
:1011E000A1E0B1E00D9111274BE351E0040F151F71
:1011F000A3E0B1E00D931C93A3E0B1E0ED91FC916D
:10120000A6E0B1E091E07ED340910601009100019B
:10121000041709F401C001C03FC1A1E0B1E00D9184
:1012200011274AE451E0040F151FA3E0B1E00D932C
:101230001C93A3E0B1E0ED91FC91A6E0B1E091E058
:1012400061D34091060100910001041709F401C027
:1012500001C022C1A1E0B1E00D91112749E551E0A3
:10126000040F151FA3E0B1E00D931C93A3E0B1E0C0
:10127000ED91FC91A6E0B1E091E044D340910601EC
:1012800000910001041709F401C001C005C1A1E0EB
:10129000B1E00D91112748E651E0040F151FA3E0BE
:1012A000B1E00D931C93A3E0B1E0ED91FC91A6E0B9
:1012B000B1E091E027D340910601009100010417AD
:1012C00009F401C001C0E8C0A1E0B1E00D9111270F
:1012D00047E751E0040F151FA3E0B1E00D931C9305
:1012E000A3E0B1E0ED91FC91A6E0B1E091E00AD37A
:1012F0004091060100910001041709F401C001C0EA
:10130000CBC0A1E0B1E00D91112746E851E0040FF8
:10131000151FA3E0B1E00D931C93A3E0B1E0ED91A4
:10132000FC91A6E0B1E091E0EDD240910601009180
:101330000001041709F401C001C0AEC0A1E0B1E092
:101340000D91112745E951E0040F151FA3E0B1E00D
:101350000D931C93A3E0B1E0ED91FC91A6E0B1E008
:1013600091E0D0D24091060100910001041709F4E8
:1013700001C001C091C0A1E0B1E00D91112744EA84
:1013800051E0040F151FA3E0B1E00D931C93A3E0FF
:10139000B1E0ED91FC91A6E0B1E091E0B3D24091D3
:1013A000060100910001041709F401C001C074C0D6
:1013B000A1E0B1E00D91112743EB51E0040F151F9F
:1013C000A3E0B1E00D931C93A3E0B1E0ED91FC919B
:1013D000A6E0B1E091E096D24091060100910001B3
:1013E000041709F401C001C057C0A1E0B1E00D919C
:1013F000112742EC51E0040F151FA3E0B1E00D935B
:101400001C93A3E0B1E0ED91FC91A6E0B1E091E086
:1014100079D24091060100910001041709F401C03E
:1014200001C03AC0A1E0B1E00D91112741ED51E0BA
:10143000040F151FA3E0B1E00D931C93A3E0B1E0EE
:10144000ED91FC91A6E0B1E091E05CD24091060103
:1014500000910001041709F401C001C01DC0A1E002
:10146000B1E00D91112740EE51E0040F151FA3E0EC
:10147000B1E00D931C93A3E0B1E0ED91FC91A6E0E7
:10148000B1E091E03FD240910601009100010417C4
:1014900009F401C07FC000C0A1E0B1E08C918F5F72
:1014A0008C9308F415CC00910F010E3010F009F068
:1014B00001C001C07DC7FAD0F7D000911101013001
:1014C00009F003C0EEE5FDE1E9D000911101023021
:1014D00009F003C0EEE6FDE1E1D000911101033017
:1014E00009F003C0E0E8FDE1D9D00091110104301A
:1014F00009F003C0E0E9FDE1D1D05E9A8AEF809364
:10150000050181E0809307017AD04A9901C0FDCF9F
:10151000CDD0CAD000911101013009F003C0E2EA38
:10152000FDE1BCD000911101023009F003C0E0EBF5
:10153000FDE1B4D000911101033009F003C0EEEBDE
:10154000FDE1ACD000911101043009F003C0ECECD6
:10155000FDE1A4D0E1E0F0E0BAD05C9AE2E0F0E096
:10156000B6D05C98A3D0E2E1F9E198D0E2E0F0E0F7
:10157000AED080910B01815080930B01EDEFF1E033
:10158000ABE0B1E091E07BE7ACD190D0E1E0F0E0FE
:101590009ED008958BD000911101013009F003C055
:1015A000EAEDFDE17BD000911101023009F003C0AA
:1015B000E8EEFDE173D000911101033009F003C0A2
:1015C000E8EFFDE16BD000911101043009F003C098
:1015D000E8E0FEE163D068D0E2E1F9E15FD05E9A35
:1015E0008AE58093050189E08093070108D04A9934
:1015F00001C0FDCFE1E0F0E06AD058D0089580E06E
:10160000809301014091070100910101041710F03E
:1016100009F013C05B9AA5E0B1E08C919927D4D072
:101620005B98A5E0B1E08C919927CED0A1E0B1E024
:101630008C918F5F8C9308F4E5CF0895ED91FC9128
:10164000EF5FFF4FFC93EE93089504D0CCD000FCE5
:101650000CD008950024E89457FF02C009D0689484
:1016600000F80BD010F80124089502D009D0089595
:10167000509540954F5F5F4F0895E89417FF089588
:10168000009510950F5F1F4F68940895A8ECB4E083
:101690008D91882311F066D0FBCF0895AED0802DB8
:1016A00011F060D0FBCF089580EC62C081E060D083
:1016B00014D080E85DC08FE7213039F08FEB223005
:1016C00021F08FE8233009F08FEC810F51C088EEB4
:1016D00093E07AD03197D9F7089583E0992774C0C1
:1016E0008AEF90E071D0259A249A239A229A219A1F
:1016F000209A289885E090E067D029982D982C981A
:101700002B9A2A9A299AEF93FF93E5E1F0E050D0C3
:10171000FF91EF91299855D0299AEF93FF93E5E136
:10172000F0E046D0FF91EF9129984BD0299AEF93A2
:10173000FF93E5E1F0E03CD0FF91EF91299841D093
:101740002A98299AEF93FF93E5E1F0E031D0FF91D9
:10175000EF91299836D088E20BD08EE009D086E050
:1017600007D00895289A829505D004D02AD00895EC
:101770002898F9CF859510F42A9A01C02A98859562
:1017800010F42B9A01C02B98859510F42C9A01C067
:101790002C98859510F42D9A01C02D98299AEF93D5
:1017A000FF93E5E1F0E004D0FF91EF9129980895CF
:1017B0003197F1F70895689462F80895E89462F813
:1017C000089581E090E000C0EF93FF93EE27E82BAF
:1017D000E92B31F0EAEFF0E03197F1F70197D1F71B
:1017E000FF91EF9108950F92B801469F8001479FA6
:1017F000100D569F100D0F900895C895319600203A
:101800000895000F111F221F331F08950095109592
:10181000209530950F5F1F4F2F4F3F4F0895019137
:1018200010810EC001911191219130810BC0019165
:10183000108117FF05C03FEF2FEF04C00081112773
:101840002227332737FF03C0E1DF8DE28D93CF934B
:10185000DF93CF92DF92EF92AA24BB24CC24DD2425
:10186000EE2440E2CAE0DD2755E093E38881890F4A
:1018700087FD9F7083FD907F891B89935A95A9F7F7
:10188000C0DFAA1CBB1CCC1CDD1CEE1C4A9551F70A
:10189000E894EFE0FF2782910ED0EB30E0F71EF0E6
:1018A00068948A2D0CD088278D93EF90DF90CF908D
:1018B000DF91CF910895982F829501D0892F8F7055
:1018C000805D26F0803309F4089568948D9308951F
:1018D000F999FECFE1BDF2BD3196089591E001C0C6
:1018E00092E07B3751F47FB7F894F2DF8D9180BDA1
:1018F000FA9AF99A9A95C9F77FBF7727089591E0E8
:1019000001C092E0E5DFF89A80B58D939A95D1F702
:1019100008955757572E4156522E344D472E434F58
:101920004D0047534D3A00002B3338360000340049
:1019300030003800330032003100370039005345A1
:10194000542F4E4153544156493D3E5131003030A1
:101950003D454E47202C2031303D534C4F00303117
:101960003D474552202C2031313D45535000202029
:10197000496E7365727420436172640056737461BA
:1019800076697465206B61727469636F0000496EDB
:101990007365727420436172642D474552200000C4
:1019A000496E7365727420436172642D45535020F3
:1019B0000000212044454D4F204558504952454490
:1019C00020210000212044454D4F20504F54454BCD
:1019D000454C2021000044454D4F20455850495268
:1019E00045442D474552000044454D4F2045585031
:1019F000495245442D455350000057726974696E31
:101A0000672043617264000056706973206B6172D5
:101A10007469636500005363687265696265204B91
:101A200061727465000047726162616E646F207458
:101A300061726A65746100004D656D6F7279206630
:101A4000756C6C3A000053706F6D696E20706F6C2E
:101A50006E3A0000537065696368657220766F6C3A
:101A60006C3A000053696E206D656D6F7269613A62
:101A7000000057726974696E6720436172643D3E6D
:101A80003031000056706973206B61727469636550
:101A90003D3E303100005363687265696265204BDA
:101AA0002E3D3E303100477261622E207461726AB1
:101AB0002E3D3E3031004B617274652065696E6663
:101AC000FC6872656E00496E73657274652074619E
:101AD000726A657461002020205475726E20436123
:101AE000726400004F62726E697465206B6172747B
:101AF00069636F0020204B617274652077656E64A6
:101B0000656E000020566F6C746565207461726AA2
:101B10006574610043617264204E6F3A00004B614E
:101B200072746963613A00004B617274654E723A77
:101B300000005461726A6574613A0000206F66208B
:101B40000000206F6420000020766F6E200020646B
:101B500065200000202020207772697474656E0073
:101B60002020202076706973616E610020206765F7
:101B700073636872696562656E0020202020677259
:101B800061626164610020205772697474696E67D4
:101B90000000202056706973756A656D000020533F
:101BA000636872656962656E000020204772616239
:101BB000616E646F000020204D6173746572204374
:101BC00061726400204D6173746572206B61727480
:101BD00069636F00202048617570742D4B617274C9
:101BE00065005461726A657461204D616573747239
:101BF0006100204F62726E69206B61727469636F5D
:101C00000000204D6173746572206B6172746963AA
:101C1000610020202020206772616261646F0000F3
:101C20002045726173696E672043617264730000BE
:101C30002042726973656D206B617274696365001F
:101C4000204B61727465206CF6736368656E0000EA
:101C500020426F7272616E646F207461726A2E002E
:101C60002066726F6D20303120746F203332000097
:101C700020206F6420303120643020333200207601
:101C80006F6E2030312062697320333200002020D3
:101C9000206465203031206120333200204361729E
:101CA00064733A203031202D203332004B6172743E
:101CB0006963653A203031202D2033320000202026
:101CC0004B617274653A2030312D3332000054611B
:101CD000726A657461733A2030312D3332002020EE
:101CE0002020202020206572617365642020000080
:101CF00020202020202020697A62726973616E653D
:101D00000000202020202020202067656CF67363CF
:101D100068740000202020202020202020626F7284
:101D20007261646F000020202020436865636B6946
:101D30006E670000202020205072657665726A610F
:101D40006D0020202020205072FC66656E0020204F
:101D50002056657269666963616E646F0000204396
:101D600061726420657863657074656400004B611E
:101D7000727469636120737072656A6574610000D2
:101D8000204B6172746520657277617274657400AE
:101D90005461726A2E206578636570747561646140
:101DA000000020202020556E6C6F636B656400007E
:101DB0002020204F646B6C656E6A656E6F0020207A
:101DC00020456E7472696567656C7400202020443C
:101DD00065737472616261646100202020436172E6
:101DE000642077726F6E67004B6172746963612063
:101DF0006E617061636E61002046616C736368653B
:101E0000204B617274650000205461726A657461D0
:081E100020657272616461003B
:00000001FF
